:020000040000FA
:1000000090286A08820741344234433444344534EA
:1000100046344734483449344A344B344C344D34F4
:100020000C140800A1004630A20016281728A20BC5
:100030001528A10B13280800A0010830A100031007
:10004000A00D851C2128050885182328A200221C44
:100050002014A10B20282008602020080800A00000
:1000600060202008A3078316051083120830A10022
:100070000510851C39288B13A01F0514A00D8518A9
:100080003F28A10B382844288316051483128B17A8
:1000900008003606E03903194F2800300800361EE4
:1000A000542836080F390800360EF0390800BB30E6
:1000B00081005C20813081070B110B1D5D28080039
:1000C0008C190800E9000611831606158312813089
:1000D00081000830E8005C20E90C031C76288316B8
:1000E000061183125A20E80B6C287C28831606150B
:1000F00083125A20E80B6C288316061183125A20AB
:10010000080083120619812857200830E8000310E0
:1001100006190314E90C5A20E80B8728690808001F
:1001200000308C00B401B501B601831203138501C0
:1001300007309F008316EF308500FF3086000000F7
:100140000615000006128F30810064008312003013
:10015000850086000000061606115530602000302C
:10016000B800B9000030BA00BB000E30BC003C3013
:10017000C0004130C1005530C2005830C3002D309E
:10018000C4004930C5004E30C6003E30C700303094
:10019000B700CA282830A1004630A200051DF62865
:1001A0008518CA28A20BCE28A10BCC28051DF6283D
:1001B0000518D628A301A0010830A100051DF628C6
:1001C00085180029051CDE28851800290C18E92847
:1001D000D6281430122083160510831205101E3005
:1001E0001220831605148312D628D6280130A100C8
:1001F000CC2806126300051DFA2864000616AF28F5
:100200001C20A400A3070319CA281C20A500A307CB
:100210001C20A600A3071C20A700A3071C20A800E1
:100220002302031DCA28A61F37291C20A900A307E3
:100230001C20AA00A3071C20AB00A3071C20AC00B5
:10024000A307261F32291C20AD00A3071C20AE00E7
:10025000A3071C20AF00A3071C20B000A3071C208D
:10026000B100A3071C20B2002302031DCA286400AA
:100270001C20B300031DCA283D292608013A031992
:1002800078292608023A0319F1298C1C6F292608BF
:10029000243A0319B8292608253A0319BA29260849
:1002A000263A0319BC292608273A0319BE2926082D
:1002B000283A0319C0292608293A0319C229260811
:1002C000083A0319C4292608343A0319C82926080C
:1002D000353A0319CA292608363A0319C6292608C9
:1002E000873A03199B292608F03A0319B029902967
:1002F0002708031992282708023A0319D229270848
:10030000113A0319122A2708123A03191F2A27083B
:10031000133A03195D2A2708153A03193A2A902936
:10032000CA2834082402031DCA280130B5008C14E1
:1003300010200030CC2927086B3A0319AC29270874
:100340008B3A0319AC292708293A0319AC29270845
:100350002A3A0319AC29CA28B5018C100130CC29DE
:100360002708340203199529B5018C100130CC29D6
:100370000B30CC290C30CC290330CC290430CC29CB
:100380000530CC290630CC290A30CC290730CC29BD
:100390000930CC290830CC29EA0000308A0001203D
:1003A0006020CA28B408031DCA28A30110302F20DA
:1003B00037082F208C302F20D0302F202308A20088
:1003C00023082F202208A30004302F20A8302F203C
:1003D0002D302F20A3302F2023082F2000302F2056
:1003E000CA282408F0393702031DCA282408B4009B
:1003F0002708B600A30110302F2034082F208C309E
:100400002F20A0302F202308A20023082F2022080D
:10041000A30024302F20A8302F203C302F20A030E4
:100420002F20EC29B408031DCA28A30110302F2067
:1004300018302F2004302F2000302F20EC293408D2
:100440002402031DCA286400A30110302F203408A1
:100450002F2000302F208030B508031D00302F20C2
:1004600023082F2000302F2035087F39003A031D44
:100470001020CA283508003A0319CA280C1CCA28BB
:10048000A30110302F2018302F2082302F20003071
:1004900049202F202308A20023082F202208A30090
:1004A000203049202F20403049202F206030492023
:1004B0002F20803049202F20EC2934082402031DEE
:1004C000CA280C10A301B50A3508023A0319852A77
:1004D0003508033A0319A72A3508043A0319EF2A05
:1004E0003508443A0319C92A3508073A0319092B74
:1004F0003508133A0319072B3508153A0319852ACD
:100500003508163A0319ED2ACA2877302F20340807
:100510002F20C0302F2040302F202308A200230896
:100520002F202208A30000302F2000302F20003081
:100530002F2000302F2000302F203B082F200130AB
:100540002F2002302F203A0E01382F20302B703010
:100550002F2034082F20C0302F2000302F202308D8
:10056000A20023082F202208A30000302F200030F3
:100570002F2000302F2000302F2000302F203B086C
:100580002F2000302F2000302F203A0E0A382F2045
:10059000302B10302F2034082F20D5302F201B3047
:1005A0002F202308A20023082F202208A300F030C8
:1005B0002F2000302F20CE302F2001302F20003070
:1005C0002F2010302F2000302F2000302F203A0E07
:1005D0000D382F200730B500302B7F30B50070303C
:1005E0002F2034082F2090302F2000302F20230878
:1005F000A20023082F202208A3003B082F20380840
:100600002F2039082F203A0E3C042F20302B7F302A
:10061000B50077302F2034082F20CD302F20400810
:100620002F202308A20023082F202208A30041081E
:100630002F2042082F2043082F2044082F20450850
:100640002F2046082F2047082F2000302F203A0E59
:100650003C042F20B50A2D2B2D2B8030B500EC2922
:1006600023082F2000302F2035087F3A031D10204B
:02067000CA2896
:02400E00E63F8B
:00000001FF
